 nframepop001

 Timestamp is 2e0f5db5 (reproducible build file hash)

 Preferred load address is 0000000180000000

 Start         Length     Name                   Class
 0001:00000000 000030e0H .text$mn                CODE
 0001:000030e0 00000036H .text$mn$00             CODE
 0001:00003116 00000092H .text$x                 CODE
 0002:00000000 00000190H .idata$5                DATA
 0002:00000190 00000038H .00cfg                  DATA
 0002:000001c8 00000008H .CRT$XCA                DATA
 0002:000001d0 00000008H .CRT$XCZ                DATA
 0002:000001d8 00000008H .CRT$XIA                DATA
 0002:000001e0 00000008H .CRT$XIC                DATA
 0002:000001e8 00000008H .CRT$XIZ                DATA
 0002:000001f0 00000008H .CRT$XLA                DATA
 0002:000001f8 00000008H .CRT$XLZ                DATA
 0002:00000200 00000008H .CRT$XPA                DATA
 0002:00000208 00000008H .CRT$XPZ                DATA
 0002:00000210 00000008H .CRT$XTA                DATA
 0002:00000218 00000008H .CRT$XTZ                DATA
 0002:00000220 00000000H .gehcont$y              DATA
 0002:00000220 00000000H .gfids$y                DATA
 0002:00000220 00001ee0H .rdata                  DATA
 0002:00002100 00000000H .rdata$CastGuardVftablesA DATA
 0002:00002100 00000000H .rdata$CastGuardVftablesC DATA
 0002:00002100 00000028H .rdata$T                DATA
 0002:00002128 000000b0H .rdata$voltmd           DATA
 0002:000021d8 00000320H .rdata$zzzdbg           DATA
 0002:000024f8 00000008H .rtc$IAA                DATA
 0002:00002500 00000008H .rtc$IZZ                DATA
 0002:00002508 00000008H .rtc$TAA                DATA
 0002:00002510 00000008H .rtc$TZZ                DATA
 0002:00002518 00000004H .tls                    DATA
 0002:0000251c 00000004H .tls$                   DATA
 0002:00002520 00000008H .tls$ZZZ                DATA
 0002:00002528 000002f8H .xdata                  DATA
 0002:00002820 00000468H .edata                  DATA
 0002:00002c88 00000064H .idata$2                DATA
 0002:00002cec 00000014H .idata$3                DATA
 0002:00002d00 00000190H .idata$4                DATA
 0002:00002e90 00000414H .idata$6                DATA
 0003:00000000 00000080H .data                   DATA
 0003:00000080 0001b3c8H .bss                    DATA
 0004:00000000 0000039cH .pdata                  DATA

  Address         Publics by Value              Rva+Base               Lib:Object

 0000:00000000       __AbsoluteZero             0000000000000000     <absolute>
 0000:00000000       ___safe_se_handler_count   0000000000000000     <absolute>
 0000:00000000       ___safe_se_handler_table   0000000000000000     <absolute>
 0000:00000000       __arm64x_extra_rfe_table   0000000000000000     <absolute>
 0000:00000000       __arm64x_extra_rfe_table_size 0000000000000000     <absolute>
 0000:00000000       __arm64x_native_entrypoint 0000000000000000     <absolute>
 0000:00000000       __arm64x_redirection_metadata 0000000000000000     <absolute>
 0000:00000000       __arm64x_redirection_metadata_count 0000000000000000     <absolute>
 0000:00000000       __dynamic_value_reloc_table 0000000000000000     <absolute>
 0000:00000000       __enclave_config           0000000000000000     <absolute>
 0000:00000000       __guard_check_icall_a64n_fptr 0000000000000000     <absolute>
 0000:00000000       __guard_eh_cont_count      0000000000000000     <absolute>
 0000:00000000       __guard_eh_cont_table      0000000000000000     <absolute>
 0000:00000000       __guard_fids_count         0000000000000000     <absolute>
 0000:00000000       __guard_fids_table         0000000000000000     <absolute>
 0000:00000000       __guard_iat_count          0000000000000000     <absolute>
 0000:00000000       __guard_iat_table          0000000000000000     <absolute>
 0000:00000000       __guard_longjmp_count      0000000000000000     <absolute>
 0000:00000000       __guard_longjmp_table      0000000000000000     <absolute>
 0000:00000000       __hybrid_auxiliary_iat     0000000000000000     <absolute>
 0000:00000000       __hybrid_auxiliary_iat_copy 0000000000000000     <absolute>
 0000:00000000       __hybrid_code_map          0000000000000000     <absolute>
 0000:00000000       __hybrid_code_map_count    0000000000000000     <absolute>
 0000:00000000       __x64_code_ranges_to_entry_points 0000000000000000     <absolute>
 0000:00000000       __x64_code_ranges_to_entry_points_count 0000000000000000     <absolute>
 0000:00000100       __guard_flags              0000000000000100     <absolute>
 0000:00000000       __ImageBase                0000000180000000     <linker-defined>
 0001:00000000       ?NewObject@JNIEnv_@@QEAAPEAV_jobject@@PEAV_jclass@@PEAU_jmethodID@@ZZ 0000000180001000 f i libnframepop001.obj
 0001:00000024       ?SetEventNotificationMode@_jvmtiEnv@@QEAA?AW4jvmtiError@@W4jvmtiEventMode@@W4jvmtiEvent@@PEAV_jobject@@ZZ 0000000180001024 f i libnframepop001.obj
 0001:0000002c       ?TranslateError@@YAPEBDW4jvmtiError@@@Z 000000018000102c f   libnframepop001.obj
 0001:000002e4       ?nsk_jni_check_exception@@YAHPEAUJNIEnv_@@QEBDH@Z 00000001800012e4 f   libnframepop001.obj
 0001:00000428       ?nsk_jni_lverify@@YAHHPEAUJNIEnv_@@HQEBDH1ZZ 0000000180001428 f   libnframepop001.obj
 0001:000004c8       Agent_Initialize           00000001800014c8 f   libnframepop001.obj
 0001:00000640       Agent_OnAttach             0000000180001640 f   libnframepop001.obj
 0001:00000640       Agent_OnLoad               0000000180001640 f   libnframepop001.obj
 0001:00000648       ExceptionCatch             0000000180001648 f   libnframepop001.obj
 0001:000007bc       FramePop                   00000001800017bc f   libnframepop001.obj
 0001:000008c8       Java_nsk_jvmti_NotifyFramePop_nframepop001_checkFrame 00000001800018c8 f   libnframepop001.obj
 0001:00000a2c       Java_nsk_jvmti_NotifyFramePop_nframepop001_getMethIds 0000000180001a2c f   libnframepop001.obj
 0001:00000b44       Java_nsk_jvmti_NotifyFramePop_nframepop001_getRes 0000000180001b44 f   libnframepop001.obj
 0001:00000b4c       Java_nsk_jvmti_NotifyFramePop_nframepop001_setFramePopNotif 0000000180001b4c f   libnframepop001.obj
 0001:00000d2c       Java_nsk_jvmti_unit_FollowReferences_FollowRefObjects_addRefToVerify 0000000180001d2c f   libnframepop001.obj
 0001:00000ee8       Java_nsk_jvmti_unit_FollowReferences_FollowRefObjects_getTag 0000000180001ee8 f   libnframepop001.obj
 0001:00000fa4       Java_nsk_jvmti_unit_FollowReferences_FollowRefObjects_resetRefsToVerify 0000000180001fa4 f   libnframepop001.obj
 0001:00000fac       Java_nsk_jvmti_unit_FollowReferences_FollowRefObjects_resetTags 0000000180001fac f   libnframepop001.obj
 0001:00000ff0       Java_nsk_jvmti_unit_FollowReferences_FollowRefObjects_setTag 0000000180001ff0 f   libnframepop001.obj
 0001:0000123c       Java_nsk_share_jvmti_ArgumentHandler_getAgentOptionsString 000000018000223c f   libnframepop001.obj
 0001:000012e8       Java_nsk_share_jvmti_DebugeeClass_checkStatus 00000001800022e8 f   libnframepop001.obj
 0001:00001370       Java_nsk_share_jvmti_DebugeeClass_resetAgentData 0000000180002370 f   libnframepop001.obj
 0001:000013d0       Java_nsk_share_jvmti_RedefineAgent_agentStatus 00000001800023d0 f   libnframepop001.obj
 0001:000013dc       Java_nsk_share_jvmti_RedefineAgent_isRedefined 00000001800023dc f   libnframepop001.obj
 0001:000013e8       Java_nsk_share_jvmti_RedefineAgent_redefineAttempted 00000001800023e8 f   libnframepop001.obj
 0001:000013f4       MA_checkStatus             00000001800023f4 f   libnframepop001.obj
 0001:00001498       __local_stdio_printf_options 0000000180002498 f i libnframepop001.obj
 0001:00001668       exitOnError                0000000180002668 f   libnframepop001.obj
 0001:0000171c       fprintf                    000000018000271c f i libnframepop001.obj
 0001:00001760       nsk_jvmti_lverify          0000000180002760 f   libnframepop001.obj
 0001:00001850       nsk_jvmti_resetAgentData   0000000180002850 f   libnframepop001.obj
 0001:000018c4       nsk_lcomplain              00000001800028c4 f   libnframepop001.obj
 0001:000018e4       nsk_ldisplay               00000001800028e4 f   libnframepop001.obj
 0001:00001904       nsk_ltrace                 0000000180002904 f   libnframepop001.obj
 0001:00001924       nsk_lvcomplain             0000000180002924 f   libnframepop001.obj
 0001:00001adc       nsk_lvdisplay              0000000180002adc f   libnframepop001.obj
 0001:00001b28       nsk_lverify                0000000180002b28 f   libnframepop001.obj
 0001:00001b84       nsk_lvtrace                0000000180002b84 f   libnframepop001.obj
 0001:00001be4       nsk_printf                 0000000180002be4 f   libnframepop001.obj
 0001:00001c0c       nsk_vprintf                0000000180002c0c f   libnframepop001.obj
 0001:00001cc0       printf                     0000000180002cc0 f i libnframepop001.obj
 0001:000021c0       __raise_securityfailure    00000001800031c0 f   MSVCRT:gs_report.obj
 0001:000021f4       __report_gsfailure         00000001800031f4 f   MSVCRT:gs_report.obj
 0001:00002434       __GSHandlerCheck           0000000180003434 f   MSVCRT:gshandler.obj
 0001:00002454       __GSHandlerCheckCommon     0000000180003454 f   MSVCRT:gshandler.obj
 0001:000024c0       __security_check_cookie    00000001800034c0 f   MSVCRT:amdsecgs.obj
 0001:00002800       _DllMainCRTStartup         0000000180003800 f   MSVCRT:dll_dllmain.obj
 0001:00002840       __scrt_acquire_startup_lock 0000000180003840 f   MSVCRT:utility.obj
 0001:0000287c       __scrt_dllmain_after_initialize_c 000000018000387c f   MSVCRT:utility.obj
 0001:000028b0       __scrt_dllmain_before_initialize_c 00000001800038b0 f   MSVCRT:utility.obj
 0001:000028c8       __scrt_dllmain_crt_thread_attach 00000001800038c8 f   MSVCRT:utility.obj
 0001:000028f0       __scrt_dllmain_crt_thread_detach 00000001800038f0 f   MSVCRT:utility.obj
 0001:00002908       __scrt_dllmain_exception_filter 0000000180003908 f   MSVCRT:utility.obj
 0001:00002968       __scrt_dllmain_uninitialize_c 0000000180003968 f   MSVCRT:utility.obj
 0001:00002998       __scrt_dllmain_uninitialize_critical 0000000180003998 f   MSVCRT:utility.obj
 0001:000029ac       __scrt_initialize_crt      00000001800039ac f   MSVCRT:utility.obj
 0001:000029f8       __scrt_initialize_onexit_tables 00000001800039f8 f   MSVCRT:utility.obj
 0001:00002a84       __scrt_is_nonwritable_in_current_image 0000000180003a84 f   MSVCRT:utility.obj
 0001:00002b1c       __scrt_release_startup_lock 0000000180003b1c f   MSVCRT:utility.obj
 0001:00002b40       __scrt_uninitialize_crt    0000000180003b40 f   MSVCRT:utility.obj
 0001:00002b6c       _onexit                    0000000180003b6c f   MSVCRT:utility.obj
 0001:00002ba8       atexit                     0000000180003ba8 f   MSVCRT:utility.obj
 0001:00002bc0       __crt_debugger_hook        0000000180003bc0 f   MSVCRT:utility_desktop.obj
 0001:00002bc8       __scrt_fastfail            0000000180003bc8 f   MSVCRT:utility_desktop.obj
 0001:00002d14       _guard_check_icall_nop     0000000180003d14 f i MSVCRT:guard_support.obj
 0001:00002d18       __security_init_cookie     0000000180003d18 f   MSVCRT:gs_support.obj
 0001:00002dc4       DllMain                    0000000180003dc4 f   MSVCRT:dll_dllmain_stub.obj
 0001:00002de8       ?__scrt_initialize_type_info@@YAXXZ 0000000180003de8 f   MSVCRT:tncleanup.obj
 0001:00002df8       ?__scrt_uninitialize_type_info@@YAXXZ 0000000180003df8 f   MSVCRT:tncleanup.obj
 0001:00002e04       __local_stdio_scanf_options 0000000180003e04 f i MSVCRT:default_local_stdio_options.obj
 0001:00002e0c       __scrt_initialize_default_local_stdio_options 0000000180003e0c f   MSVCRT:default_local_stdio_options.obj
 0001:00002e28       __scrt_get_dyn_tls_init_callback 0000000180003e28 f   MSVCRT:dyn_tls_init.obj
 0001:00002e30       _RTC_Initialize            0000000180003e30 f   MSVCRT:initsect.obj
 0001:00002e6c       _RTC_Terminate             0000000180003e6c f   MSVCRT:initsect.obj
 0001:00002ea8       __isa_available_init       0000000180003ea8 f   MSVCRT:cpu_disp.obj
 0001:00003054       _get_startup_argv_mode     0000000180004054 f   MSVCRT:argv_mode.obj
 0001:0000305c       __scrt_is_ucrt_dll_in_use  000000018000405c f   MSVCRT:ucrt_detection.obj
 0001:00003070       memcpy                     0000000180004070 f   vcruntime:VCRUNTIME140.dll
 0001:00003076       memset                     0000000180004076 f   vcruntime:VCRUNTIME140.dll
 0001:0000307c       strchr                     000000018000407c f   vcruntime:VCRUNTIME140.dll
 0001:00003082       __C_specific_handler       0000000180004082 f   vcruntime:VCRUNTIME140.dll
 0001:00003088       __std_type_info_destroy_list 0000000180004088 f   vcruntime:VCRUNTIME140.dll
 0001:0000308e       strlen                     000000018000408e f   ucrt:api-ms-win-crt-string-l1-1-0.dll
 0001:00003094       _initterm                  0000000180004094 f   ucrt:api-ms-win-crt-runtime-l1-1-0.dll
 0001:0000309a       _initterm_e                000000018000409a f   ucrt:api-ms-win-crt-runtime-l1-1-0.dll
 0001:000030a0       _seh_filter_dll            00000001800040a0 f   ucrt:api-ms-win-crt-runtime-l1-1-0.dll
 0001:000030a6       _configure_narrow_argv     00000001800040a6 f   ucrt:api-ms-win-crt-runtime-l1-1-0.dll
 0001:000030ac       _initialize_narrow_environment 00000001800040ac f   ucrt:api-ms-win-crt-runtime-l1-1-0.dll
 0001:000030b2       _initialize_onexit_table   00000001800040b2 f   ucrt:api-ms-win-crt-runtime-l1-1-0.dll
 0001:000030b8       _register_onexit_function  00000001800040b8 f   ucrt:api-ms-win-crt-runtime-l1-1-0.dll
 0001:000030be       _execute_onexit_table      00000001800040be f   ucrt:api-ms-win-crt-runtime-l1-1-0.dll
 0001:000030c4       _crt_atexit                00000001800040c4 f   ucrt:api-ms-win-crt-runtime-l1-1-0.dll
 0001:000030ca       _cexit                     00000001800040ca f   ucrt:api-ms-win-crt-runtime-l1-1-0.dll
 0001:000030d0       __acrt_initialize          00000001800040d0 f   MSVCRT:ucrt_stubs.obj
 0001:000030d0       __acrt_thread_attach       00000001800040d0 f   MSVCRT:ucrt_stubs.obj
 0001:000030d0       __acrt_thread_detach       00000001800040d0 f   MSVCRT:ucrt_stubs.obj
 0001:000030d0       __acrt_uninitialize        00000001800040d0 f   MSVCRT:ucrt_stubs.obj
 0001:000030d0       __acrt_uninitialize_critical 00000001800040d0 f   MSVCRT:ucrt_stubs.obj
 0001:000030d0       __scrt_stub_for_acrt_initialize 00000001800040d0 f   MSVCRT:ucrt_stubs.obj
 0001:000030d0       __scrt_stub_for_acrt_thread_attach 00000001800040d0 f   MSVCRT:ucrt_stubs.obj
 0001:000030d0       __scrt_stub_for_acrt_thread_detach 00000001800040d0 f   MSVCRT:ucrt_stubs.obj
 0001:000030d0       __scrt_stub_for_acrt_uninitialize 00000001800040d0 f   MSVCRT:ucrt_stubs.obj
 0001:000030d0       __scrt_stub_for_acrt_uninitialize_critical 00000001800040d0 f   MSVCRT:ucrt_stubs.obj
 0001:000030d0       __vcrt_initialize          00000001800040d0 f   MSVCRT:ucrt_stubs.obj
 0001:000030d0       __vcrt_thread_attach       00000001800040d0 f   MSVCRT:ucrt_stubs.obj
 0001:000030d0       __vcrt_thread_detach       00000001800040d0 f   MSVCRT:ucrt_stubs.obj
 0001:000030d0       __vcrt_uninitialize        00000001800040d0 f   MSVCRT:ucrt_stubs.obj
 0001:000030d0       __vcrt_uninitialize_critical 00000001800040d0 f   MSVCRT:ucrt_stubs.obj
 0001:000030d4       __scrt_stub_for_is_c_termination_complete 00000001800040d4 f   MSVCRT:ucrt_stubs.obj
 0001:000030d4       _is_c_termination_complete 00000001800040d4 f   MSVCRT:ucrt_stubs.obj
 0001:000030f0       _guard_dispatch_icall_nop  00000001800040f0 f   MSVCRT:guard_dispatch.obj
 0001:00003110       _guard_xfg_dispatch_icall_nop 0000000180004110 f   MSVCRT:guard_xfg_dispatch.obj
 0002:00000000       __imp_RtlCaptureContext    0000000180005000     kernel32:KERNEL32.dll
 0002:00000008       __imp_RtlLookupFunctionEntry 0000000180005008     kernel32:KERNEL32.dll
 0002:00000010       __imp_RtlVirtualUnwind     0000000180005010     kernel32:KERNEL32.dll
 0002:00000018       __imp_UnhandledExceptionFilter 0000000180005018     kernel32:KERNEL32.dll
 0002:00000020       __imp_SetUnhandledExceptionFilter 0000000180005020     kernel32:KERNEL32.dll
 0002:00000028       __imp_GetCurrentProcess    0000000180005028     kernel32:KERNEL32.dll
 0002:00000030       __imp_TerminateProcess     0000000180005030     kernel32:KERNEL32.dll
 0002:00000038       __imp_IsProcessorFeaturePresent 0000000180005038     kernel32:KERNEL32.dll
 0002:00000040       __imp_CloseHandle          0000000180005040     kernel32:KERNEL32.dll
 0002:00000048       __imp_InitializeCriticalSectionAndSpinCount 0000000180005048     kernel32:KERNEL32.dll
 0002:00000050       __imp_DeleteCriticalSection 0000000180005050     kernel32:KERNEL32.dll
 0002:00000058       __imp_CreateEventW         0000000180005058     kernel32:KERNEL32.dll
 0002:00000060       __imp_GetModuleHandleW     0000000180005060     kernel32:KERNEL32.dll
 0002:00000068       __imp_GetProcAddress       0000000180005068     kernel32:KERNEL32.dll
 0002:00000070       __imp_IsDebuggerPresent    0000000180005070     kernel32:KERNEL32.dll
 0002:00000078       __imp_QueryPerformanceCounter 0000000180005078     kernel32:KERNEL32.dll
 0002:00000080       __imp_GetCurrentProcessId  0000000180005080     kernel32:KERNEL32.dll
 0002:00000088       __imp_GetCurrentThreadId   0000000180005088     kernel32:KERNEL32.dll
 0002:00000090       __imp_GetSystemTimeAsFileTime 0000000180005090     kernel32:KERNEL32.dll
 0002:00000098       __imp_DisableThreadLibraryCalls 0000000180005098     kernel32:KERNEL32.dll
 0002:000000a0       __imp_InitializeSListHead  00000001800050a0     kernel32:KERNEL32.dll
 0002:000000a8       \177KERNEL32_NULL_THUNK_DATA 00000001800050a8     kernel32:KERNEL32.dll
 0002:000000b0       __imp_memcpy               00000001800050b0     vcruntime:VCRUNTIME140.dll
 0002:000000b8       __imp_memset               00000001800050b8     vcruntime:VCRUNTIME140.dll
 0002:000000c0       __imp_strchr               00000001800050c0     vcruntime:VCRUNTIME140.dll
 0002:000000c8       __imp___C_specific_handler 00000001800050c8     vcruntime:VCRUNTIME140.dll
 0002:000000d0       __imp___std_type_info_destroy_list 00000001800050d0     vcruntime:VCRUNTIME140.dll
 0002:000000d8       \177VCRUNTIME140_NULL_THUNK_DATA 00000001800050d8     vcruntime:VCRUNTIME140.dll
 0002:000000e0       __imp__errno               00000001800050e0     ucrt:api-ms-win-crt-runtime-l1-1-0.dll
 0002:000000e8       __imp_exit                 00000001800050e8     ucrt:api-ms-win-crt-runtime-l1-1-0.dll
 0002:000000f0       __imp__cexit               00000001800050f0     ucrt:api-ms-win-crt-runtime-l1-1-0.dll
 0002:000000f8       __imp__crt_atexit          00000001800050f8     ucrt:api-ms-win-crt-runtime-l1-1-0.dll
 0002:00000100       __imp__execute_onexit_table 0000000180005100     ucrt:api-ms-win-crt-runtime-l1-1-0.dll
 0002:00000108       __imp__register_onexit_function 0000000180005108     ucrt:api-ms-win-crt-runtime-l1-1-0.dll
 0002:00000110       __imp__initialize_onexit_table 0000000180005110     ucrt:api-ms-win-crt-runtime-l1-1-0.dll
 0002:00000118       __imp__initialize_narrow_environment 0000000180005118     ucrt:api-ms-win-crt-runtime-l1-1-0.dll
 0002:00000120       __imp__configure_narrow_argv 0000000180005120     ucrt:api-ms-win-crt-runtime-l1-1-0.dll
 0002:00000128       __imp__seh_filter_dll      0000000180005128     ucrt:api-ms-win-crt-runtime-l1-1-0.dll
 0002:00000130       __imp__initterm_e          0000000180005130     ucrt:api-ms-win-crt-runtime-l1-1-0.dll
 0002:00000138       __imp__initterm            0000000180005138     ucrt:api-ms-win-crt-runtime-l1-1-0.dll
 0002:00000140       \177api-ms-win-crt-runtime-l1-1-0_NULL_THUNK_DATA 0000000180005140     ucrt:api-ms-win-crt-runtime-l1-1-0.dll
 0002:00000148       __imp___acrt_iob_func      0000000180005148     ucrt:api-ms-win-crt-stdio-l1-1-0.dll
 0002:00000150       __imp_fflush               0000000180005150     ucrt:api-ms-win-crt-stdio-l1-1-0.dll
 0002:00000158       __imp___stdio_common_vsprintf 0000000180005158     ucrt:api-ms-win-crt-stdio-l1-1-0.dll
 0002:00000160       __imp___stdio_common_vfprintf 0000000180005160     ucrt:api-ms-win-crt-stdio-l1-1-0.dll
 0002:00000168       \177api-ms-win-crt-stdio-l1-1-0_NULL_THUNK_DATA 0000000180005168     ucrt:api-ms-win-crt-stdio-l1-1-0.dll
 0002:00000170       __imp__strdup              0000000180005170     ucrt:api-ms-win-crt-string-l1-1-0.dll
 0002:00000170       __imp_strdup               0000000180005170     ucrt:api-ms-win-crt-string-l1-1-0.dll
 0002:00000178       __imp_strlen               0000000180005178     ucrt:api-ms-win-crt-string-l1-1-0.dll
 0002:00000180       __imp_strncpy              0000000180005180     ucrt:api-ms-win-crt-string-l1-1-0.dll
 0002:00000188       \177api-ms-win-crt-string-l1-1-0_NULL_THUNK_DATA 0000000180005188     ucrt:api-ms-win-crt-string-l1-1-0.dll
 0002:00000190       __guard_check_icall_fptr   0000000180005190     MSVCRT:guard_support.obj
 0002:00000198       __guard_xfg_check_icall_fptr 0000000180005198     MSVCRT:guard_support.obj
 0002:000001a0       __guard_dispatch_icall_fptr 00000001800051a0     MSVCRT:guard_support.obj
 0002:000001a8       __guard_xfg_dispatch_icall_fptr 00000001800051a8     MSVCRT:guard_support.obj
 0002:000001b0       __guard_xfg_table_dispatch_icall_fptr 00000001800051b0     MSVCRT:guard_support.obj
 0002:000001b8       __castguard_check_failure_os_handled_fptr 00000001800051b8     MSVCRT:guard_support.obj
 0002:000001c0       __guard_memcpy_fptr        00000001800051c0     vcruntime:softmemtag.obj
 0002:000001c8       __xc_a                     00000001800051c8     MSVCRT:initializers.obj
 0002:000001d0       __xc_z                     00000001800051d0     MSVCRT:initializers.obj
 0002:000001d8       __xi_a                     00000001800051d8     MSVCRT:initializers.obj
 0002:000001e8       __xi_z                     00000001800051e8     MSVCRT:initializers.obj
 0002:000001f0       __xl_a                     00000001800051f0     MSVCRT:tlssup.obj
 0002:000001f8       __xl_z                     00000001800051f8     MSVCRT:tlssup.obj
 0002:00000200       __xp_a                     0000000180005200     MSVCRT:initializers.obj
 0002:00000208       __xp_z                     0000000180005208     MSVCRT:initializers.obj
 0002:00000210       __xt_a                     0000000180005210     MSVCRT:initializers.obj
 0002:00000218       __xt_z                     0000000180005218     MSVCRT:initializers.obj
 0002:00000220       g_refKindStr               0000000180005220     libnframepop001.obj
 0002:000003d0       ??_C@_09BPLDFGCI@unknown_0@ 00000001800053d0     libnframepop001.obj
 0002:000003e0       ??_C@_0BL@FPNMECJD@JVMTI_HEAP_REFERENCE_CLASS@ 00000001800053e0     libnframepop001.obj
 0002:00000400       ??_C@_0BL@FKGKKLNM@JVMTI_HEAP_REFERENCE_FIELD@ 0000000180005400     libnframepop001.obj
 0002:00000420       ??_C@_0CD@CAEHCFJF@JVMTI_HEAP_REFERENCE_ARRAY_ELEM@ 0000000180005420     libnframepop001.obj
 0002:00000448       ??_C@_0CC@DNEBMCNK@JVMTI_HEAP_REFERENCE_CLASS_LOAD@ 0000000180005448     libnframepop001.obj
 0002:00000470       ??_C@_0BN@CJMIPEBB@JVMTI_HEAP_REFERENCE_SIGNERS@ 0000000180005470     libnframepop001.obj
 0002:00000490       ??_C@_0CH@HBOIDPEB@JVMTI_HEAP_REFERENCE_PROTECTION@ 0000000180005490     libnframepop001.obj
 0002:000004b8       ??_C@_0BP@MDKGDGKL@JVMTI_HEAP_REFERENCE_INTERFACE@ 00000001800054b8     libnframepop001.obj
 0002:000004d8       ??_C@_0CC@JJMIHNJH@JVMTI_HEAP_REFERENCE_STATIC_FIE@ 00000001800054d8     libnframepop001.obj
 0002:00000500       ??_C@_0CD@IDHEEGID@JVMTI_HEAP_REFERENCE_CONSTANT_P@ 0000000180005500     libnframepop001.obj
 0002:00000528       ??_C@_0CA@EFFCHNG@JVMTI_HEAP_REFERENCE_SUPERCLASS@ 0000000180005528     libnframepop001.obj
 0002:00000548       ??_C@_0L@PCDFHGCJ@unknown_11@ 0000000180005548     libnframepop001.obj
 0002:00000558       ??_C@_0L@NJBICFOK@unknown_12@ 0000000180005558     libnframepop001.obj
 0002:00000568       ??_C@_0L@MAADBEKL@unknown_13@ 0000000180005568     libnframepop001.obj
 0002:00000578       ??_C@_0L@IPECICGM@unknown_14@ 0000000180005578     libnframepop001.obj
 0002:00000588       ??_C@_0L@JGFJLDCN@unknown_15@ 0000000180005588     libnframepop001.obj
 0002:00000598       ??_C@_0L@LNHEOAOO@unknown_16@ 0000000180005598     libnframepop001.obj
 0002:000005a8       ??_C@_0L@KEGPNBKP@unknown_17@ 00000001800055a8     libnframepop001.obj
 0002:000005b8       ??_C@_0L@CDPHMNGA@unknown_18@ 00000001800055b8     libnframepop001.obj
 0002:000005c8       ??_C@_0L@DKOMPMCB@unknown_19@ 00000001800055c8     libnframepop001.obj
 0002:000005d8       ??_C@_0L@OJGIPJDB@unknown_20@ 00000001800055d8     libnframepop001.obj
 0002:000005e8       ??_C@_0CA@KAOFNDEM@JVMTI_HEAP_REFERENCE_JNI_GLOBAL@ 00000001800055e8     libnframepop001.obj
 0002:00000608       ??_C@_0CC@HPFAJBK@JVMTI_HEAP_REFERENCE_SYSTEM_CLA@ 0000000180005608     libnframepop001.obj
 0002:00000630       ??_C@_0BN@FDEGFOHC@JVMTI_HEAP_REFERENCE_MONITOR@ 0000000180005630     libnframepop001.obj
 0002:00000650       ??_C@_0CB@HKIBCMAJ@JVMTI_HEAP_REFERENCE_STACK_LOCA@ 0000000180005650     libnframepop001.obj
 0002:00000678       ??_C@_0BP@EAACMMOE@JVMTI_HEAP_REFERENCE_JNI_LOCAL@ 0000000180005678     libnframepop001.obj
 0002:00000698       ??_C@_0BM@IJDEOGOE@JVMTI_HEAP_REFERENCE_THREAD@ 0000000180005698     libnframepop001.obj
 0002:000006b8       ??_C@_0BL@EDGPPKC@JVMTI_HEAP_REFERENCE_OTHER@ 00000001800056b8     libnframepop001.obj
 0002:000006d4       ??_C@_04BCJPDBDA@Code@     00000001800056d4     libnframepop001.obj
 0002:000006e0       ??_C@_0BA@OCLMCFKC@LineNumberTable@ 00000001800056e0     libnframepop001.obj
 0002:000006f0       ??_C@_0BD@CPAEPILC@LocalVariableTable@ 00000001800056f0     libnframepop001.obj
 0002:00000708       ??_C@_0BH@NMBDNHBD@LocalVariableTypeTable@ 0000000180005708     libnframepop001.obj
 0002:00000720       ??_C@_0O@HIHEEDNJ@StackMapTable@ 0000000180005720     libnframepop001.obj
 0002:00000730       ??_C@_0L@HCDIAMJG@?9?5?$CFs?0?5?$CFd?3?5@ 0000000180005730     libnframepop001.obj
 0002:00000740       ??_C@_0JI@HLPECLFI@?$CD?5?4?4?4?6?$CD?5ERROR?3?5too?5many?5complai@ 0000000180005740     libnframepop001.obj
 0002:000007e0       ??_C@_0ED@JNEKCCOB@The?5following?5fake?5exception?5st@ 00000001800057e0     libnframepop001.obj
 0002:00000828       ??_C@_0CN@FCNMDFBH@nsk?4share?4Fake_Exception_for_RU@ 0000000180005828     libnframepop001.obj
 0002:00000858       ??_C@_08PGFFNAEI@?$CI?$CFs?3?$CFd?$CJ?5@ 0000000180005858     libnframepop001.obj
 0002:00000868       ??_C@_0DP@IENMAEGI@s?2test?2hotspot?2jtreg?2vmTestbase@ 0000000180005868     libnframepop001.obj
 0002:000008a8       ??_C@_0BL@NDJLFFJB@?7at?5nsk_lvcomplain?$CI?$CFs?3?$CFd?$CJ?6@ 00000001800058a8     libnframepop001.obj
 0002:000008c8       ??_C@_0BC@JOOKAFKF@?$CD?5ERROR?3?5?$CFs?0?5?$CFd?3?5@ 00000001800058c8     libnframepop001.obj
 0002:000008e0       ??_C@_09KJEAHMEH@?$CD?5ERROR?3?5@ 00000001800058e0     libnframepop001.obj
 0002:000008ec       ??_C@_02GPIOPFAK@?$DO?$DO@ 00000001800058ec     libnframepop001.obj
 0002:000008f0       ??_C@_02FODMEDOG@?$DM?$DM@ 00000001800058f0     libnframepop001.obj
 0002:000008f4       ??_C@_02DJGKEECL@?4?4@     00000001800058f4     libnframepop001.obj
 0002:000008f8       ??_C@_0O@CJPGJOAF@?9?5?$CFs?0?5?$CFd?3?5?$CFs?5@ 00000001800058f8     libnframepop001.obj
 0002:00000908       ??_C@_0CB@IAKPDOIC@?$CD?5?5?5verified?5assertion?5is?5FALSE@ 0000000180005908     libnframepop001.obj
 0002:00000930       ??_C@_0CO@LGONDEPD@stdout?3?5fflush?5failed?5?9?5err?$DN?$CFd?5@ 0000000180005930     libnframepop001.obj
 0002:00000960       ??_C@_0CO@KBGKJPBD@stderr?3?5fflush?5failed?5?9?5err?$DN?$CFd?5@ 0000000180005960     libnframepop001.obj
 0002:00000990       ??_C@_0BB@JCNMKLLK@JVMTI_ERROR_NONE@ 0000000180005990     libnframepop001.obj
 0002:000009a8       ??_C@_0BL@LDIMKLPH@JVMTI_ERROR_INVALID_THREAD@ 00000001800059a8     libnframepop001.obj
 0002:000009c8       ??_C@_0CB@PJFPAIKJ@JVMTI_ERROR_INVALID_THREAD_GROU@ 00000001800059c8     libnframepop001.obj
 0002:000009f0       ??_C@_0BN@LLMKHMNF@JVMTI_ERROR_INVALID_PRIORITY@ 00000001800059f0     libnframepop001.obj
 0002:00000a10       ??_C@_0CB@MBOFKAGB@JVMTI_ERROR_THREAD_NOT_SUSPENDE@ 0000000180005a10     libnframepop001.obj
 0002:00000a38       ??_C@_0BN@FABOLPBI@JVMTI_ERROR_THREAD_SUSPENDED@ 0000000180005a38     libnframepop001.obj
 0002:00000a58       ??_C@_0BN@FDGNOBJM@JVMTI_ERROR_THREAD_NOT_ALIVE@ 0000000180005a58     libnframepop001.obj
 0002:00000a78       ??_C@_0BL@GOBIFKNJ@JVMTI_ERROR_INVALID_OBJECT@ 0000000180005a78     libnframepop001.obj
 0002:00000a98       ??_C@_0BK@FCMAJPPC@JVMTI_ERROR_INVALID_CLASS@ 0000000180005a98     libnframepop001.obj
 0002:00000ab8       ??_C@_0BP@IKLLBKEB@JVMTI_ERROR_CLASS_NOT_PREPARED@ 0000000180005ab8     libnframepop001.obj
 0002:00000ad8       ??_C@_0BN@KLPPLKG@JVMTI_ERROR_INVALID_METHODID@ 0000000180005ad8     libnframepop001.obj
 0002:00000af8       ??_C@_0BN@BCEKOKND@JVMTI_ERROR_INVALID_LOCATION@ 0000000180005af8     libnframepop001.obj
 0002:00000b18       ??_C@_0BM@DFDGPME@JVMTI_ERROR_INVALID_FIELDID@ 0000000180005b18     libnframepop001.obj
 0002:00000b38       ??_C@_0BL@NELIEPEC@JVMTI_ERROR_NO_MORE_FRAMES@ 0000000180005b38     libnframepop001.obj
 0002:00000b58       ??_C@_0BJ@BDBECFDM@JVMTI_ERROR_OPAQUE_FRAME@ 0000000180005b58     libnframepop001.obj
 0002:00000b78       ??_C@_0BK@MIIFNLOB@JVMTI_ERROR_TYPE_MISMATCH@ 0000000180005b78     libnframepop001.obj
 0002:00000b98       ??_C@_0BJ@HPCAOILC@JVMTI_ERROR_INVALID_SLOT@ 0000000180005b98     libnframepop001.obj
 0002:00000bb8       ??_C@_0BG@CHILOPNI@JVMTI_ERROR_DUPLICATE@ 0000000180005bb8     libnframepop001.obj
 0002:00000bd0       ??_C@_0BG@DIEMLHKM@JVMTI_ERROR_NOT_FOUND@ 0000000180005bd0     libnframepop001.obj
 0002:00000be8       ??_C@_0BM@NHMCKHOB@JVMTI_ERROR_INVALID_MONITOR@ 0000000180005be8     libnframepop001.obj
 0002:00000c08       ??_C@_0BO@PPEDAJGL@JVMTI_ERROR_NOT_MONITOR_OWNER@ 0000000180005c08     libnframepop001.obj
 0002:00000c28       ??_C@_0BG@FCAIPEID@JVMTI_ERROR_INTERRUPT@ 0000000180005c28     libnframepop001.obj
 0002:00000c40       ??_C@_0CB@EGDBNKOI@JVMTI_ERROR_INVALID_CLASS_FORMA@ 0000000180005c40     libnframepop001.obj
 0002:00000c68       ??_C@_0CG@DGKOGIAL@JVMTI_ERROR_CIRCULAR_CLASS_DEFI@ 0000000180005c68     libnframepop001.obj
 0002:00000c90       ??_C@_0BP@ICEALPKC@JVMTI_ERROR_FAILS_VERIFICATION@ 0000000180005c90     libnframepop001.obj
 0002:00000cb0       ??_C@_0DC@JDACLMIO@JVMTI_ERROR_UNSUPPORTED_REDEFIN@ 0000000180005cb0     libnframepop001.obj
 0002:00000ce8       ??_C@_0DE@GKDKNOMJ@JVMTI_ERROR_UNSUPPORTED_REDEFIN@ 0000000180005ce8     libnframepop001.obj
 0002:00000d20       ??_C@_0BO@LAFKIOG@JVMTI_ERROR_INVALID_TYPESTATE@ 0000000180005d20     libnframepop001.obj
 0002:00000d40       ??_C@_0DH@INDGCLLB@JVMTI_ERROR_UNSUPPORTED_REDEFIN@ 0000000180005d40     libnframepop001.obj
 0002:00000d78       ??_C@_0DE@NHEOMMGI@JVMTI_ERROR_UNSUPPORTED_REDEFIN@ 0000000180005d78     libnframepop001.obj
 0002:00000db0       ??_C@_0CA@EKPNJOEP@JVMTI_ERROR_UNSUPPORTED_VERSION@ 0000000180005db0     libnframepop001.obj
 0002:00000dd0       ??_C@_0BN@OFFMAHHL@JVMTI_ERROR_NAMES_DONT_MATCH@ 0000000180005dd0     libnframepop001.obj
 0002:00000df0       ??_C@_0DN@HHBBLAKE@JVMTI_ERROR_UNSUPPORTED_REDEFIN@ 0000000180005df0     libnframepop001.obj
 0002:00000e30       ??_C@_0DO@HMBGBGNA@JVMTI_ERROR_UNSUPPORTED_REDEFIN@ 0000000180005e30     libnframepop001.obj
 0002:00000e70       ??_C@_0BP@PBECGKHJ@JVMTI_ERROR_UNMODIFIABLE_CLASS@ 0000000180005e70     libnframepop001.obj
 0002:00000e90       ??_C@_0BK@CANILEHF@JVMTI_ERROR_NOT_AVAILABLE@ 0000000180005e90     libnframepop001.obj
 0002:00000eb0       ??_C@_0CE@INJKMEFK@JVMTI_ERROR_MUST_POSSESS_CAPABI@ 0000000180005eb0     libnframepop001.obj
 0002:00000ed8       ??_C@_0BJ@LBFPFPDM@JVMTI_ERROR_NULL_POINTER@ 0000000180005ed8     libnframepop001.obj
 0002:00000ef8       ??_C@_0BP@CHJPNNEM@JVMTI_ERROR_ABSENT_INFORMATION@ 0000000180005ef8     libnframepop001.obj
 0002:00000f18       ??_C@_0BP@OMFMNLC@JVMTI_ERROR_INVALID_EVENT_TYPE@ 0000000180005f18     libnframepop001.obj
 0002:00000f38       ??_C@_0BN@BIBNPHHO@JVMTI_ERROR_ILLEGAL_ARGUMENT@ 0000000180005f38     libnframepop001.obj
 0002:00000f58       ??_C@_0BK@KKNDHDCE@JVMTI_ERROR_NATIVE_METHOD@ 0000000180005f58     libnframepop001.obj
 0002:00000f78       ??_C@_0BK@PMKCFHAE@JVMTI_ERROR_OUT_OF_MEMORY@ 0000000180005f78     libnframepop001.obj
 0002:00000f98       ??_C@_0BK@NNJBDMNB@JVMTI_ERROR_ACCESS_DENIED@ 0000000180005f98     libnframepop001.obj
 0002:00000fb8       ??_C@_0BI@GHECLMNC@JVMTI_ERROR_WRONG_PHASE@ 0000000180005fb8     libnframepop001.obj
 0002:00000fd0       ??_C@_0BF@OLIHJOII@JVMTI_ERROR_INTERNAL@ 0000000180005fd0     libnframepop001.obj
 0002:00000fe8       ??_C@_0BO@EOHGKJHI@JVMTI_ERROR_UNATTACHED_THREAD@ 0000000180005fe8     libnframepop001.obj
 0002:00001008       ??_C@_0CA@LKHFDACL@JVMTI_ERROR_INVALID_ENVIRONMENT@ 0000000180006008     libnframepop001.obj
 0002:00001028       ??_C@_0BA@MMFHLOKK@?$DMunknown?5error?$DO@ 0000000180006028     libnframepop001.obj
 0002:00001038       ??_C@_0CF@CBHOKDB@throwable?5?$DN?5jni?9?$DOExceptionOccur@ 0000000180006038     libnframepop001.obj
 0002:00001060       ??_C@_03OFAPEBGM@?$CFs?6@  0000000180006060     libnframepop001.obj
 0002:00001068       ??_C@_0DM@LPIGEGNJ@s?2test?2hotspot?2jtreg?2vmTestbase@ 0000000180006068     libnframepop001.obj
 0002:000010a8       ??_C@_0CC@NFCNPEPK@Exception?5in?5JNI?5call?5?$CIcleared?$CJ@ 00000001800060a8     libnframepop001.obj
 0002:000010d0       ??_C@_0BJ@IBAKFIKF@jni?9?$DOExceptionDescribe?$CI?$CJ@ 00000001800060d0     libnframepop001.obj
 0002:000010f0       ??_C@_0BG@GGKALKMH@jni?9?$DOExceptionClear?$CI?$CJ@ 00000001800060f0     libnframepop001.obj
 0002:00001108       ??_C@_0CF@JMGFGJLJ@?$CD?5?5?5verified?5JNI?5assertion?5is?5F@ 0000000180006108     libnframepop001.obj
 0002:00001130       ??_C@_0CB@MLNJNCLJ@?5?5jvmti?5error?3?5code?$DN?$CFd?0?5name?$DN?$CFs@ 0000000180006130     libnframepop001.obj
 0002:00001158       ??_C@_0CD@OHBGDKMK@?$CD?5?5?5jvmti?5error?3?5code?$DN?$CFd?0?5name?$DN@ 0000000180006158     libnframepop001.obj
 0002:00001180       ??_C@_0CG@JNNCGPHB@?$CD?5?5?5error?5expected?3?5code?$DN?$CFd?0?5na@ 0000000180006180     libnframepop001.obj
 0002:000011b0       ??_C@_0EB@IMGKPCGE@?$CIstr_obj?5?$DN?5jni?9?$DONewStringUTF?$CIco@ 00000001800061b0     libnframepop001.obj
 0002:00001200       ??_C@_0EA@HFOGGBCC@s?2test?2hotspot?2jtreg?2vmTestbase@ 0000000180006200     libnframepop001.obj
 0002:00001240       ??_C@_0CK@GNODJBHO@?$CIResumeThread?$CJ?5unexpected?5error@ 0000000180006240     libnframepop001.obj
 0002:00001270       ??_C@_0CL@KLNIBDFF@?$CISuspendThread?$CJ?5unexpected?5erro@ 0000000180006270     libnframepop001.obj
 0002:0000129c       ??_C@_05KKCIMGE@error@     000000018000629c     libnframepop001.obj
 0002:000012b0       ??_C@_0EA@PNBCDMOA@s?2test?2hotspot?2jtreg?2vmTestbase@ 00000001800062b0     libnframepop001.obj
 0002:000012f0       ??_C@_0DI@ILAHDLMP@?$CI?$CKagentThreadProc?$CJ?$CIjvmti_env?0?5a@ 00000001800062f0     libnframepop001.obj
 0002:00001328       ??_C@_0BD@KDBALNLB@JVMTI?5agent?5thread@ 0000000180006328     libnframepop001.obj
 0002:00001340       ??_C@_0BB@NOKBFPFO@java?1lang?1Thread@ 0000000180006340     libnframepop001.obj
 0002:00001354       ??_C@_06FALKBLGB@?$DMinit?$DO@ 0000000180006354     libnframepop001.obj
 0002:00001360       ??_C@_0BG@IKDDPPGD@?$CILjava?1lang?1String?$DL?$CJV@ 0000000180006360     libnframepop001.obj
 0002:00001380       ??_C@_0EB@IFJBFEKC@?$CIthreadClass?5?$DN?5jni_env?9?$DOFindCla@ 0000000180006380     libnframepop001.obj
 0002:000013d0       ??_C@_0GF@FGFIBKKL@?$CIthreadCtor?5?$DN?5jni_env?9?$DOGetMetho@ 00000001800063d0     libnframepop001.obj
 0002:00001438       ??_C@_0DN@NCPDJLOG@?$CIthreadName?5?$DN?5jni_env?9?$DONewStrin@ 0000000180006438     libnframepop001.obj
 0002:00001480       ??_C@_0FE@PFKODBGC@?$CIthreadObject?5?$DN?5jni_env?9?$DONewObj@ 0000000180006480     libnframepop001.obj
 0002:000014e0       ??_C@_0ED@HOBAHHJI@?$CIthreadGlobalRef?5?$DN?5jni_env?9?$DONew@ 00000001800064e0     libnframepop001.obj
 0002:00001530       ??_C@_0FN@HNJJAHFC@jvmti_env?9?$DORunAgentThread?$CIagent@ 0000000180006530     libnframepop001.obj
 0002:00001590       ??_C@_0EA@MOJDNKDF@Debuggee?5status?5sync?5aborted?5be@ 0000000180006590     libnframepop001.obj
 0002:000015d0       ??_C@_0EA@EEOEJAEN@status?5?$DN?5syncDebuggeeStatus?$CIjni@ 00000001800065d0     libnframepop001.obj
 0002:00001610       ??_C@_0BL@JBCFNBMB@nsk_jvmti_resetAgentData?$CI?$CJ@ 0000000180006610     libnframepop001.obj
 0002:00001630       ??_C@_0EL@LPBEELIP@s?2test?2hotspot?2jtreg?2vmTestbase@ 0000000180006630     libnframepop001.obj
 0002:00001680       ??_C@_0CK@JDAMFDMJ@jvmti?9?$DOSetTag?$CIo?0?5tag?$CJ?5?$DN?$DN?5JVMTI_@ 0000000180006680     libnframepop001.obj
 0002:000016b0       ??_C@_0CC@DAMNHKNI@Can?8t?5set?5tag?5?$CFli?5for?5object?5?$CFl@ 00000001800066b0     libnframepop001.obj
 0002:000016d8       ??_C@_0DL@HAJPNKEF@jvmti?9?$DOGetObjectHashCode?$CIo?0?5?$CGha@ 00000001800066d8     libnframepop001.obj
 0002:00001718       ??_C@_0BL@JFPIEOBF@Can?8t?5get?5hash?5object?5?$CFlx?6@ 0000000180006718     libnframepop001.obj
 0002:00001738       ??_C@_0BG@DICPHBKN@setTag?3?5?$CF08x?5?$DM?9?5?$CF?53li@ 0000000180006738     libnframepop001.obj
 0002:00001750       ??_C@_0DH@FCEEBDMJ@?$CIs?5?$DN?5jni?9?$DOGetStringUTFChars?$CIsIn@ 0000000180006750     libnframepop001.obj
 0002:00001788       ??_C@_0BJ@OKKGHDCN@Can?8t?5get?5string?5at?5?$CF?$CDp?6@ 0000000180006788     libnframepop001.obj
 0002:000017a8       ??_C@_0BP@EKFLGGFJ@Can?8t?5get?5string?5at?5?$CF?$CDp?3?5null?6@ 00000001800067a8     libnframepop001.obj
 0002:000017c8       ??_C@_06ICODBHCL@?5?1?1?5?$CFs@ 00000001800067c8     libnframepop001.obj
 0002:000017d0       ??_C@_0DB@KGFPLEGO@?$CIr?5?$DN?5jvmti?9?$DOGetTag?$CIo?0?5?$CGtag?$CJ?$CJ?5?$DN?$DN@ 00000001800067d0     libnframepop001.obj
 0002:00001808       ??_C@_0CO@PDAGBCGJ@Can?8t?5GetTag?5for?5object?5?$CFlx?4?5Re@ 0000000180006808     libnframepop001.obj
 0002:00001838       ??_C@_0CH@HPEODOHC@TEST_BUG?3?5Max?4?5number?5of?5refs?5r@ 0000000180006838     libnframepop001.obj
 0002:00001860       ??_C@_0DI@PHFCABIM@?$CIr?5?$DN?5jvmti?9?$DOGetTag?$CIfrom?0?5?$CGtagFr@ 0000000180006860     libnframepop001.obj
 0002:00001898       ??_C@_0DI@MDEGFNKD@TEST_BUG?3?5Can?8t?5GetTag?5for?5obje@ 0000000180006898     libnframepop001.obj
 0002:000018d0       ??_C@_0DE@MLELJAHM@?$CIr?5?$DN?5jvmti?9?$DOGetTag?$CIto?0?5?$CGtagTo?$CJ?$CJ@ 00000001800068d0     libnframepop001.obj
 0002:00001904       ??_C@_03GAEACAIP@?$CI?$CJV@ 0000000180006904     libnframepop001.obj
 0002:00001908       ??_C@_0DF@BMPOKPHD@?$CIGetMethodDeclaringClass?$CJ?5unexp@ 0000000180006908     libnframepop001.obj
 0002:00001940       ??_C@_0CN@PFBBHEKD@?$CIGetLocalInt?$CDpop?$CJ?5unexpected?5er@ 0000000180006940     libnframepop001.obj
 0002:00001970       ??_C@_0CP@POGHHDKP@?$CIGetLocalInt?$CDcatch?$CJ?5unexpected?5@ 0000000180006970     libnframepop001.obj
 0002:000019a0       ??_C@_0DC@JLPHMNPA@?$CINotifyFramePop?$CDcatch?$CJ?5unexpect@ 00000001800069a0     libnframepop001.obj
 0002:000019d8       ??_C@_0CJ@KCDEKOCJ@Wrong?5result?5of?5a?5valid?5call?5to@ 00000001800069d8     libnframepop001.obj
 0002:00001a08       ??_C@_0DG@LAJPGIIE@?$CIGetPotentialCapabilities?$CJ?5unex@ 0000000180006a08     libnframepop001.obj
 0002:00001a40       ??_C@_0CN@LKPEOJPO@?$CIAddCapabilities?$CJ?5unexpected?5er@ 0000000180006a40     libnframepop001.obj
 0002:00001a70       ??_C@_0CN@BCCBOHCH@?$CIGetCapabilities?$CJ?5unexpected?5er@ 0000000180006a70     libnframepop001.obj
 0002:00001aa0       ??_C@_0CP@IMINGNLL@?$CISetEventCallbacks?$CJ?5unexpected?5@ 0000000180006aa0     libnframepop001.obj
 0002:00001ad0       ??_C@_0DO@FMOGDJIP@Warning?3?5FramePop?5or?5ExceptionC@ 0000000180006ad0     libnframepop001.obj
 0002:00001b10       ??_C@_0CJ@GNEHIJOM@Warning?3?5GetLocalInt?5is?5not?5imp@ 0000000180006b10     libnframepop001.obj
 0002:00001b40       ??_C@_0CM@FEKJDMLD@Warning?3?5suspend?1resume?5is?5not?5@ 0000000180006b40     libnframepop001.obj
 0002:00001b70       ??_C@_0CL@EPIEADBE@Failed?5to?5enable?5FRAME_POP?5even@ 0000000180006b70     libnframepop001.obj
 0002:00001b9c       ??_C@_04PFANPMCN@?$CII?$CJV@ 0000000180006b9c     libnframepop001.obj
 0002:00001ba4       ??_C@_06MADNOIIM@meth01@   0000000180006ba4     libnframepop001.obj
 0002:00001bb0       ??_C@_0BN@CGJIILDC@Cannot?5find?5method?5?$CCmeth01?$CC?6@ 0000000180006bb0     libnframepop001.obj
 0002:00001bd0       ??_C@_06OLBALLEP@meth02@   0000000180006bd0     libnframepop001.obj
 0002:00001bd8       ??_C@_0BN@DECNCENM@Cannot?5find?5method?5?$CCmeth02?$CC?6@ 0000000180006bd8     libnframepop001.obj
 0002:00001bf8       ??_C@_0DB@KABMDOAM@Failed?5to?5enable?5EXCEPTION_CATC@ 0000000180006bf8     libnframepop001.obj
 0002:00001c30       ??_C@_0CH@IMODGNEA@nsk?1jvmti?1NotifyFramePop?1nframe@ 0000000180006c30     libnframepop001.obj
 0002:00001c58       ??_C@_0DL@OPPDCDOM@Cannot?5find?5nsk?4jvmti?4NotifyFra@ 0000000180006c58     libnframepop001.obj
 0002:00001c94       ??_C@_03LGMJKEGG@run@      0000000180006c94     libnframepop001.obj
 0002:00001c98       ??_C@_0BK@JAIPPBHD@Cannot?5find?5method?5?$CCrun?$CC?6@ 0000000180006c98     libnframepop001.obj
 0002:00001cb8       ??_C@_0CJ@INBPLIKC@?$CIGetLocalInt?$CJ?5unexpected?5error?3@ 0000000180006cb8     libnframepop001.obj
 0002:00001ce8       ??_C@_0CM@DJHCDKC@?$CINotifyFramePop?$CJ?5unexpected?5err@ 0000000180006ce8     libnframepop001.obj
 0002:00001d18       ??_C@_0CO@FOBLCPAJ@Point?5?$CFd?3?5thread?5is?5not?5the?5sam@ 0000000180006d18     libnframepop001.obj
 0002:00001d48       ??_C@_0CN@OKDHIKG@Point?5?$CFd?3?5class?5is?5not?5the?5same@ 0000000180006d48     libnframepop001.obj
 0002:00001d78       ??_C@_0DC@KHELENDI@Point?5?$CFd?3?5method?5ID?5expected?3?50@ 0000000180006d78     libnframepop001.obj
 0002:00001db0       ??_C@_0DL@HFKCEGMA@Point?5?$CFd?3?5was_poped_by_exceptio@ 0000000180006db0     libnframepop001.obj
 0002:00001df0       ??_C@_0CK@ILCBECHB@Point?5?$CFd?3?5local?5expected?3?5?$CFd?0?5a@ 0000000180006df0     libnframepop001.obj
 0002:00001e30       ??_C@_1EC@JIJBPKFM@?$AAa?$AAp?$AAi?$AA?9?$AAm?$AAs?$AA?9?$AAw?$AAi?$AAn?$AA?9?$AAc?$AAo?$AAr?$AAe@ 0000000180006e30     MSVCRT:thread_safe_statics.obj
 0002:00001e78       ??_C@_1BK@MGMFAEKH@?$AAk?$AAe?$AAr?$AAn?$AAe?$AAl?$AA3?$AA2?$AA?4?$AAd?$AAl?$AAl@ 0000000180006e78     MSVCRT:thread_safe_statics.obj
 0002:00001e98       ??_C@_0BJ@JEBJOJFJ@SleepConditionVariableCS@ 0000000180006e98     MSVCRT:thread_safe_statics.obj
 0002:00001eb8       ??_C@_0BJ@PGPPEPCC@WakeAllConditionVariable@ 0000000180006eb8     MSVCRT:thread_safe_statics.obj
 0002:00001ed8       _pDefaultRawDllMain        0000000180006ed8     MSVCRT:dll_dllmain.obj
 0002:00001ed8       _pRawDllMain               0000000180006ed8     MSVCRT:dll_dllmain.obj
 0002:00001ee0       __xmm@ffffffffffffffffffffffffffffffff 0000000180006ee0     MSVCRT:utility.obj
 0002:00001ef0       _load_config_used          0000000180006ef0     MSVCRT:loadcfg.obj
 0002:00002100       _tls_used                  0000000180007100     MSVCRT:tlssup.obj
 0002:00002128       __volatile_metadata        0000000180007128     <linker-defined>
 0002:000024f8       __rtc_iaa                  00000001800074f8     MSVCRT:initsect.obj
 0002:00002500       __rtc_izz                  0000000180007500     MSVCRT:initsect.obj
 0002:00002508       __rtc_taa                  0000000180007508     MSVCRT:initsect.obj
 0002:00002510       __rtc_tzz                  0000000180007510     MSVCRT:initsect.obj
 0002:00002518       _tls_start                 0000000180007518     MSVCRT:tlssup.obj
 0002:0000251c       _Init_thread_epoch         000000018000751c     MSVCRT:thread_safe_statics.obj
 0002:00002520       _tls_end                   0000000180007520     MSVCRT:tlssup.obj
 0002:00002c88       __IMPORT_DESCRIPTOR_KERNEL32 0000000180007c88     kernel32:KERNEL32.dll
 0002:00002c9c       __IMPORT_DESCRIPTOR_VCRUNTIME140 0000000180007c9c     vcruntime:VCRUNTIME140.dll
 0002:00002cb0       __IMPORT_DESCRIPTOR_api-ms-win-crt-runtime-l1-1-0 0000000180007cb0     ucrt:api-ms-win-crt-runtime-l1-1-0.dll
 0002:00002cc4       __IMPORT_DESCRIPTOR_api-ms-win-crt-stdio-l1-1-0 0000000180007cc4     ucrt:api-ms-win-crt-stdio-l1-1-0.dll
 0002:00002cd8       __IMPORT_DESCRIPTOR_api-ms-win-crt-string-l1-1-0 0000000180007cd8     ucrt:api-ms-win-crt-string-l1-1-0.dll
 0002:00002cec       __NULL_IMPORT_DESCRIPTOR   0000000180007cec     kernel32:KERNEL32.dll
 0003:00000030       _Init_global_epoch         0000000180009030     MSVCRT:thread_safe_statics.obj
 0003:00000040       __security_cookie          0000000180009040     MSVCRT:gs_cookie.obj
 0003:00000048       __security_cookie_complement 0000000180009048     MSVCRT:gs_cookie.obj
 0003:00000050       __scrt_native_dllmain_reason 0000000180009050     MSVCRT:utility.obj
 0003:00000058       __isa_available            0000000180009058     MSVCRT:cpu_disp.obj
 0003:0000005c       __isa_enabled              000000018000905c     MSVCRT:cpu_disp.obj
 0003:00000060       __memset_fast_string_threshold 0000000180009060     MSVCRT:cpu_disp.obj
 0003:00000068       __memset_nt_threshold      0000000180009068     MSVCRT:cpu_disp.obj
 0003:00000070       __scrt_ucrt_dll_is_in_use  0000000180009070     MSVCRT:ucrt_stubs.obj
 0003:00000080       g_wrongHeapCallbacks       0000000180009080     libnframepop001.obj
 0003:00000100       g_szTagInfo                0000000180009100     libnframepop001.obj
 0003:00002040       g_tagFlags                 000000018000b040     libnframepop001.obj
 0003:00002428       g_refsToVerifyCnt          000000018000b428     libnframepop001.obj
 0003:0000242c       g_fakeUserData             000000018000b42c     libnframepop001.obj
 0003:00002430       g_tagVisitCount            000000018000b430     libnframepop001.obj
 0003:000033d0       g_refsToVerify             000000018000c3d0     libnframepop001.obj
 0003:0001aad0       g_userDataError            0000000180023ad0     libnframepop001.obj
 0003:0001ae00       ?_OptionsStorage@?1??__local_stdio_printf_options@@9@4_KA 0000000180023e00     libnframepop001.obj
 0003:0001b3c8       _tls_index                 00000001800243c8     MSVCRT:tlssup.obj
 0003:0001b3d0       __scrt_current_native_startup_state 00000001800243d0     MSVCRT:utility.obj
 0003:0001b3d8       __scrt_native_startup_lock 00000001800243d8     MSVCRT:utility.obj
 0003:0001b418       __scrt_debugger_hook_flag  0000000180024418     MSVCRT:utility_desktop.obj
 0003:0001b420       ?__type_info_root_node@@3U__type_info_node@@A 0000000180024420     MSVCRT:tncleanup.obj
 0003:0001b430       ?_OptionsStorage@?1??__local_stdio_scanf_options@@9@4_KA 0000000180024430     MSVCRT:default_local_stdio_options.obj
 0003:0001b438       __favor                    0000000180024438     MSVCRT:cpu_disp.obj
 0003:0001b440       __dyn_tls_init_callback    0000000180024440     <common>

 entry point at        0001:00002800

 Static symbols

 0000:fffd9000       .debug$S                   0000000180000000     nframepop001.exp
 0000:fffd9000       .debug$S                   0000000180000000     vcruntime:VCRUNTIME140.dll
 0000:fffd9000       .debug$S                   0000000180000000     vcruntime:VCRUNTIME140.dll
 0000:fffd9000       .debug$S                   0000000180000000     vcruntime:VCRUNTIME140.dll
 0000:fffd9000       .debug$S                   0000000180000000     vcruntime:VCRUNTIME140.dll
 0000:fffd9000       .debug$S                   0000000180000000     vcruntime:VCRUNTIME140.dll
 0000:fffd9000       .debug$S                   0000000180000000     vcruntime:VCRUNTIME140.dll
 0000:fffd9000       .debug$S                   0000000180000000     vcruntime:VCRUNTIME140.dll
 0000:fffd9000       .debug$S                   0000000180000000     ucrt:api-ms-win-crt-convert-l1-1-0.dll
 0002:ffffb000       .idata$6                   0000000180000000     ucrt:api-ms-win-crt-convert-l1-1-0.dll
 0000:fffd9000       .debug$S                   0000000180000000     ucrt:api-ms-win-crt-heap-l1-1-0.dll
 0000:fffd9000       .debug$S                   0000000180000000     ucrt:api-ms-win-crt-heap-l1-1-0.dll
 0000:fffd9000       .debug$S                   0000000180000000     ucrt:api-ms-win-crt-heap-l1-1-0.dll
 0000:fffd9000       .debug$S                   0000000180000000     ucrt:api-ms-win-crt-heap-l1-1-0.dll
 0002:ffffb000       .idata$6                   0000000180000000     ucrt:api-ms-win-crt-heap-l1-1-0.dll
 0000:fffd9000       .debug$S                   0000000180000000     ucrt:api-ms-win-crt-runtime-l1-1-0.dll
 0000:fffd9000       .debug$S                   0000000180000000     ucrt:api-ms-win-crt-runtime-l1-1-0.dll
 0000:fffd9000       .debug$S                   0000000180000000     ucrt:api-ms-win-crt-runtime-l1-1-0.dll
 0000:fffd9000       .debug$S                   0000000180000000     ucrt:api-ms-win-crt-runtime-l1-1-0.dll
 0000:fffd9000       .debug$S                   0000000180000000     ucrt:api-ms-win-crt-runtime-l1-1-0.dll
 0000:fffd9000       .debug$S                   0000000180000000     ucrt:api-ms-win-crt-runtime-l1-1-0.dll
 0000:fffd9000       .debug$S                   0000000180000000     ucrt:api-ms-win-crt-runtime-l1-1-0.dll
 0000:fffd9000       .debug$S                   0000000180000000     ucrt:api-ms-win-crt-runtime-l1-1-0.dll
 0000:fffd9000       .debug$S                   0000000180000000     ucrt:api-ms-win-crt-runtime-l1-1-0.dll
 0000:fffd9000       .debug$S                   0000000180000000     ucrt:api-ms-win-crt-runtime-l1-1-0.dll
 0000:fffd9000       .debug$S                   0000000180000000     ucrt:api-ms-win-crt-runtime-l1-1-0.dll
 0000:fffd9000       .debug$S                   0000000180000000     ucrt:api-ms-win-crt-runtime-l1-1-0.dll
 0000:fffd9000       .debug$S                   0000000180000000     ucrt:api-ms-win-crt-runtime-l1-1-0.dll
 0000:fffd9000       .debug$S                   0000000180000000     ucrt:api-ms-win-crt-runtime-l1-1-0.dll
 0000:fffd9000       .debug$S                   0000000180000000     ucrt:api-ms-win-crt-runtime-l1-1-0.dll
 0000:fffd9000       .debug$S                   0000000180000000     ucrt:api-ms-win-crt-runtime-l1-1-0.dll
 0000:fffd9000       .debug$S                   0000000180000000     ucrt:api-ms-win-crt-stdio-l1-1-0.dll
 0000:fffd9000       .debug$S                   0000000180000000     ucrt:api-ms-win-crt-stdio-l1-1-0.dll
 0000:fffd9000       .debug$S                   0000000180000000     ucrt:api-ms-win-crt-stdio-l1-1-0.dll
 0000:fffd9000       .debug$S                   0000000180000000     ucrt:api-ms-win-crt-stdio-l1-1-0.dll
 0000:fffd9000       .debug$S                   0000000180000000     ucrt:api-ms-win-crt-stdio-l1-1-0.dll
 0000:fffd9000       .debug$S                   0000000180000000     ucrt:api-ms-win-crt-stdio-l1-1-0.dll
 0000:fffd9000       .debug$S                   0000000180000000     ucrt:api-ms-win-crt-stdio-l1-1-0.dll
 0000:fffd9000       .debug$S                   0000000180000000     ucrt:api-ms-win-crt-stdio-l1-1-0.dll
 0000:fffd9000       .debug$S                   0000000180000000     ucrt:api-ms-win-crt-stdio-l1-1-0.dll
 0000:fffd9000       .debug$S                   0000000180000000     ucrt:api-ms-win-crt-stdio-l1-1-0.dll
 0000:fffd9000       .debug$S                   0000000180000000     ucrt:api-ms-win-crt-string-l1-1-0.dll
 0000:fffd9000       .debug$S                   0000000180000000     ucrt:api-ms-win-crt-string-l1-1-0.dll
 0000:fffd9000       .debug$S                   0000000180000000     ucrt:api-ms-win-crt-string-l1-1-0.dll
 0000:fffd9000       .debug$S                   0000000180000000     ucrt:api-ms-win-crt-string-l1-1-0.dll
 0000:fffd9000       .debug$S                   0000000180000000     ucrt:api-ms-win-crt-string-l1-1-0.dll
 0000:fffd9000       .debug$S                   0000000180000000     ucrt:api-ms-win-crt-string-l1-1-0.dll
 0000:fffd9000       .debug$S                   0000000180000000     ucrt:api-ms-win-crt-string-l1-1-0.dll
 0000:fffd9000       .debug$S                   0000000180000000     ucrt:api-ms-win-crt-string-l1-1-0.dll
 0000:fffd9000       .debug$S                   0000000180000000     kernel32:KERNEL32.dll
 0000:fffd9000       .debug$S                   0000000180000000     kernel32:KERNEL32.dll
 0000:fffd9000       .debug$S                   0000000180000000     kernel32:KERNEL32.dll
 0000:fffd9000       .debug$S                   0000000180000000     kernel32:KERNEL32.dll
 0000:fffd9000       .debug$S                   0000000180000000     kernel32:KERNEL32.dll
 0000:fffd9000       .debug$S                   0000000180000000     kernel32:KERNEL32.dll
 0000:fffd9000       .debug$S                   0000000180000000     kernel32:KERNEL32.dll
 0000:fffd9000       .debug$S                   0000000180000000     kernel32:KERNEL32.dll
 0000:fffd9000       .debug$S                   0000000180000000     kernel32:KERNEL32.dll
 0000:fffd9000       .debug$S                   0000000180000000     kernel32:KERNEL32.dll
 0000:fffd9000       .debug$S                   0000000180000000     kernel32:KERNEL32.dll
 0000:fffd9000       .debug$S                   0000000180000000     kernel32:KERNEL32.dll
 0000:fffd9000       .debug$S                   0000000180000000     kernel32:KERNEL32.dll
 0000:fffd9000       .debug$S                   0000000180000000     kernel32:KERNEL32.dll
 0000:fffd9000       .debug$S                   0000000180000000     kernel32:KERNEL32.dll
 0000:fffd9000       .debug$S                   0000000180000000     kernel32:KERNEL32.dll
 0000:fffd9000       .debug$S                   0000000180000000     kernel32:KERNEL32.dll
 0000:fffd9000       .debug$S                   0000000180000000     kernel32:KERNEL32.dll
 0000:fffd9000       .debug$S                   0000000180000000     kernel32:KERNEL32.dll
 0000:fffd9000       .debug$S                   0000000180000000     kernel32:KERNEL32.dll
 0000:fffd9000       .debug$S                   0000000180000000     kernel32:KERNEL32.dll
 0000:fffd9000       .debug$S                   0000000180000000     kernel32:KERNEL32.dll
 0000:fffd9000       .debug$S                   0000000180000000     kernel32:KERNEL32.dll
 0000:fffd9000       .debug$S                   0000000180000000     kernel32:KERNEL32.dll
 0000:fffd9000       .debug$S                   0000000180000000     kernel32:KERNEL32.dll
 0000:fffd9000       .debug$S                   0000000180000000     kernel32:KERNEL32.dll
 0000:fffd9000       .debug$S                   0000000180000000     kernel32:KERNEL32.dll
 0000:fffd9000       .debug$S                   0000000180000000     kernel32:KERNEL32.dll
 0001:000014a0       addRefToVerify             00000001800024a0 f   libnframepop001.obj
 0001:00001514       agentThreadWrapper         0000000180002514 f   libnframepop001.obj
 0001:000016ec       file_basename              00000001800026ec f   libnframepop001.obj
 0001:00001d14       startAgentThreadWrapper    0000000180002d14 f   libnframepop001.obj
 0001:00002040       syncDebuggeeStatus         0000000180003040 f   libnframepop001.obj
 0001:000022c8       capture_previous_context   00000001800032c8 f   MSVCRT:gs_report.obj
 0001:0000233c       ?__scrt_initialize_thread_safe_statics@@YAHXZ 000000018000333c f   MSVCRT:thread_safe_statics.obj
 0001:0000240c       ?__scrt_uninitialize_thread_safe_statics@@YAXXZ 000000018000340c f   MSVCRT:thread_safe_statics.obj
 0001:000024b0       $$000000                   00000001800034b0     MSVCRT:amdsecgs.obj
 0001:000024e0       ?dllmain_crt_dispatch@@YAHQEAUHINSTANCE__@@KQEAX@Z 00000001800034e0 f   MSVCRT:dll_dllmain.obj
 0001:00002530       ?dllmain_crt_process_attach@@YAHQEAUHINSTANCE__@@QEAX@Z 0000000180003530 f   MSVCRT:dll_dllmain.obj
 0001:00002648       ?dllmain_crt_process_detach@@YAH_N@Z 0000000180003648 f   MSVCRT:dll_dllmain.obj
 0001:000026cc       ?dllmain_dispatch@@YAHQEAUHINSTANCE__@@KQEAX@Z 00000001800036cc f   MSVCRT:dll_dllmain.obj
 0001:000030e0       $$000000                   00000001800040e0     MSVCRT:guard_dispatch.obj
 0001:00003100       $$000000                   0000000180004100     MSVCRT:guard_xfg_dispatch.obj
 0001:00003116       ?fin$0@?0??dllmain_crt_process_attach@@YAHQEAUHINSTANCE__@@QEAX@Z@4HA 0000000180004116 f   MSVCRT:dll_dllmain.obj
 0001:0000312d       ?fin$0@?0??dllmain_crt_process_detach@@YAH_N@Z@4HA 000000018000412d f   MSVCRT:dll_dllmain.obj
 0001:00003146       ?fin$1@?0??dllmain_crt_process_detach@@YAH_N@Z@4HA 0000000180004146 f   MSVCRT:dll_dllmain.obj
 0001:0000315a       ?filt$0@?0??dllmain_dispatch@@YAHQEAUHINSTANCE__@@KQEAX@Z@4HA 000000018000415a f   MSVCRT:dll_dllmain.obj
 0001:00003190       __scrt_is_nonwritable_in_current_image$filt$0 0000000180004190 f   MSVCRT:utility.obj
 0002:000001e0       ?__scrt_initialize_tss_var@@3P6AHXZEA 00000001800051e0     MSVCRT:thread_safe_statics.obj
 0002:00000300       ?opcLengths@@3QBEB         0000000180005300     libnframepop001.obj
 0002:00001e20       GS_ExceptionPointers       0000000180006e20     MSVCRT:gs_report.obj
 0002:00002528       $unwind$fprintf            0000000180007528     libnframepop001.obj
 0002:00002534       $unwind$printf             0000000180007534     libnframepop001.obj
 0002:00002540       $unwind$?NewObject@JNIEnv_@@QEAAPEAV_jobject@@PEAV_jclass@@PEAU_jmethodID@@ZZ 0000000180007540     libnframepop001.obj
 0002:00002540       $unwind$nsk_lcomplain      0000000180007540     libnframepop001.obj
 0002:00002540       $unwind$nsk_ldisplay       0000000180007540     libnframepop001.obj
 0002:00002548       $unwind$nsk_lvdisplay      0000000180007548     libnframepop001.obj
 0002:00002548       $unwind$_RTC_Initialize    0000000180007548     MSVCRT:initsect.obj
 0002:00002548       $unwind$_RTC_Terminate     0000000180007548     MSVCRT:initsect.obj
 0002:00002548       $unwind$?__scrt_initialize_thread_safe_statics@@YAHXZ 0000000180007548     MSVCRT:thread_safe_statics.obj
 0002:00002554       $unwind$nsk_lvcomplain     0000000180007554     libnframepop001.obj
 0002:0000256c       $unwind$nsk_ltrace         000000018000756c     libnframepop001.obj
 0002:0000256c       $unwind$__report_gsfailure 000000018000756c     MSVCRT:gs_report.obj
 0002:00002574       $unwind$Agent_Initialize   0000000180007574     libnframepop001.obj
 0002:00002574       $unwind$nsk_lvtrace        0000000180007574     libnframepop001.obj
 0002:00002574       $unwind$__raise_securityfailure 0000000180007574     MSVCRT:gs_report.obj
 0002:00002574       $unwind$__scrt_initialize_crt 0000000180007574     MSVCRT:utility.obj
 0002:00002574       $unwind$__scrt_initialize_onexit_tables 0000000180007574     MSVCRT:utility.obj
 0002:00002574       $unwind$__scrt_release_startup_lock 0000000180007574     MSVCRT:utility.obj
 0002:00002574       $unwind$__scrt_uninitialize_crt 0000000180007574     MSVCRT:utility.obj
 0002:00002574       $unwind$_onexit            0000000180007574     MSVCRT:utility.obj
 0002:0000257c       $unwind$nsk_lverify        000000018000757c     libnframepop001.obj
 0002:0000258c       $unwind$Java_nsk_jvmti_NotifyFramePop_nframepop001_setFramePopNotif 000000018000758c     libnframepop001.obj
 0002:0000258c       $unwind$nsk_vprintf        000000018000758c     libnframepop001.obj
 0002:0000259c       $unwind$nsk_printf         000000018000759c     libnframepop001.obj
 0002:000025a4       $unwind$?nsk_jni_lverify@@YAHHPEAUJNIEnv_@@HQEBDH1ZZ 00000001800075a4     libnframepop001.obj
 0002:000025b8       $unwind$?nsk_jni_check_exception@@YAHPEAUJNIEnv_@@QEBDH@Z 00000001800075b8     libnframepop001.obj
 0002:000025d4       $unwind$Java_nsk_jvmti_unit_FollowReferences_FollowRefObjects_resetTags 00000001800075d4     libnframepop001.obj
 0002:000025d4       $unwind$addRefToVerify     00000001800075d4     libnframepop001.obj
 0002:000025d4       $unwind$nsk_jvmti_resetAgentData 00000001800075d4     libnframepop001.obj
 0002:000025d4       $unwind$__scrt_initialize_default_local_stdio_options 00000001800075d4     MSVCRT:default_local_stdio_options.obj
 0002:000025d4       $unwind$?dllmain_crt_dispatch@@YAHQEAUHINSTANCE__@@KQEAX@Z 00000001800075d4     MSVCRT:dll_dllmain.obj
 0002:000025d4       $unwind$DllMain            00000001800075d4     MSVCRT:dll_dllmain_stub.obj
 0002:000025d4       $unwind$__GSHandlerCheck   00000001800075d4     MSVCRT:gshandler.obj
 0002:000025d4       $unwind$?__scrt_uninitialize_thread_safe_statics@@YAXXZ 00000001800075d4     MSVCRT:thread_safe_statics.obj
 0002:000025d4       $unwind$__scrt_acquire_startup_lock 00000001800075d4     MSVCRT:utility.obj
 0002:000025d4       $unwind$__scrt_dllmain_after_initialize_c 00000001800075d4     MSVCRT:utility.obj
 0002:000025d4       $unwind$__scrt_dllmain_before_initialize_c 00000001800075d4     MSVCRT:utility.obj
 0002:000025d4       $unwind$__scrt_dllmain_crt_thread_attach 00000001800075d4     MSVCRT:utility.obj
 0002:000025d4       $unwind$__scrt_dllmain_crt_thread_detach 00000001800075d4     MSVCRT:utility.obj
 0002:000025d4       $unwind$__scrt_dllmain_uninitialize_c 00000001800075d4     MSVCRT:utility.obj
 0002:000025d4       $unwind$__scrt_dllmain_uninitialize_critical 00000001800075d4     MSVCRT:utility.obj
 0002:000025d4       $unwind$atexit             00000001800075d4     MSVCRT:utility.obj
 0002:000025dc       $unwind$nsk_jvmti_lverify  00000001800075dc     libnframepop001.obj
 0002:000025f0       $unwind$exitOnError        00000001800075f0     libnframepop001.obj
 0002:00002600       $unwind$Java_nsk_share_jvmti_ArgumentHandler_getAgentOptionsString 0000000180007600     libnframepop001.obj
 0002:00002614       $unwind$Java_nsk_jvmti_unit_FollowReferences_FollowRefObjects_getTag 0000000180007614     libnframepop001.obj
 0002:00002614       $unwind$Java_nsk_share_jvmti_DebugeeClass_checkStatus 0000000180007614     libnframepop001.obj
 0002:00002614       $unwind$agentThreadWrapper 0000000180007614     libnframepop001.obj
 0002:00002624       $unwind$startAgentThreadWrapper 0000000180007624     libnframepop001.obj
 0002:00002640       $unwind$syncDebuggeeStatus 0000000180007640     libnframepop001.obj
 0002:00002640       $unwind$__scrt_dllmain_exception_filter 0000000180007640     MSVCRT:utility.obj
 0002:00002654       $unwind$Java_nsk_share_jvmti_DebugeeClass_resetAgentData 0000000180007654     libnframepop001.obj
 0002:0000265c       $unwind$MA_checkStatus     000000018000765c     libnframepop001.obj
 0002:00002670       $unwind$Java_nsk_jvmti_unit_FollowReferences_FollowRefObjects_setTag 0000000180007670     libnframepop001.obj
 0002:00002688       $unwind$Java_nsk_jvmti_unit_FollowReferences_FollowRefObjects_addRefToVerify 0000000180007688     libnframepop001.obj
 0002:000026a4       $unwind$ExceptionCatch     00000001800076a4     libnframepop001.obj
 0002:000026a4       $unwind$FramePop           00000001800076a4     libnframepop001.obj
 0002:000026bc       $unwind$Java_nsk_jvmti_NotifyFramePop_nframepop001_getMethIds 00000001800076bc     libnframepop001.obj
 0002:000026bc       $unwind$_DllMainCRTStartup 00000001800076bc     MSVCRT:dll_dllmain.obj
 0002:000026cc       $unwind$Java_nsk_jvmti_NotifyFramePop_nframepop001_checkFrame 00000001800076cc     libnframepop001.obj
 0002:000026dc       $unwind$capture_previous_context 00000001800076dc     MSVCRT:gs_report.obj
 0002:000026e8       $unwind$__GSHandlerCheckCommon 00000001800076e8     MSVCRT:gshandler.obj
 0002:000026f0       $xdatasym                  00000001800076f0     MSVCRT:amdsecgs.obj
 0002:000026f4       $unwind$?dllmain_crt_process_attach@@YAHQEAUHINSTANCE__@@QEAX@Z 00000001800076f4     MSVCRT:dll_dllmain.obj
 0002:00002730       $unwind$?fin$0@?0??dllmain_crt_process_attach@@YAHQEAUHINSTANCE__@@QEAX@Z@4HA 0000000180007730     MSVCRT:dll_dllmain.obj
 0002:00002730       $unwind$?fin$0@?0??dllmain_crt_process_detach@@YAH_N@Z@4HA 0000000180007730     MSVCRT:dll_dllmain.obj
 0002:00002730       $unwind$?fin$1@?0??dllmain_crt_process_detach@@YAH_N@Z@4HA 0000000180007730     MSVCRT:dll_dllmain.obj
 0002:00002738       $unwind$?dllmain_crt_process_detach@@YAH_N@Z 0000000180007738     MSVCRT:dll_dllmain.obj
 0002:0000278c       $unwind$?dllmain_dispatch@@YAHQEAUHINSTANCE__@@KQEAX@Z 000000018000778c     MSVCRT:dll_dllmain.obj
 0002:000027b4       $unwind$?filt$0@?0??dllmain_dispatch@@YAHQEAUHINSTANCE__@@KQEAX@Z@4HA 00000001800077b4     MSVCRT:dll_dllmain.obj
 0002:000027bc       $unwind$__scrt_is_nonwritable_in_current_image 00000001800077bc     MSVCRT:utility.obj
 0002:000027dc       $unwind$__scrt_is_nonwritable_in_current_image$filt$0 00000001800077dc     MSVCRT:utility.obj
 0002:000027e4       $unwind$__scrt_fastfail    00000001800077e4     MSVCRT:utility_desktop.obj
 0002:000027f4       $unwind$__security_init_cookie 00000001800077f4     MSVCRT:gs_support.obj
 0002:00002800       $unwind$__isa_available_init 0000000180007800     MSVCRT:cpu_disp.obj
 0002:00002810       $xdatasym                  0000000180007810     MSVCRT:guard_dispatch.obj
 0002:00002818       $xdatasym                  0000000180007818     MSVCRT:guard_xfg_dispatch.obj
 0002:00002820       .edata                     0000000180007820     nframepop001.exp
 0002:00002848       rgpv                       0000000180007848     nframepop001.exp
 0002:00002890       rgszName                   0000000180007890     nframepop001.exp
 0002:000028d8       rgwOrd                     00000001800078d8     nframepop001.exp
 0002:000028fc       szName                     00000001800078fc     nframepop001.exp
 0002:0000290d       $N00001                    000000018000790d     nframepop001.exp
 0002:0000291c       $N00002                    000000018000791c     nframepop001.exp
 0002:00002929       $N00003                    0000000180007929     nframepop001.exp
 0002:0000295f       $N00004                    000000018000795f     nframepop001.exp
 0002:00002995       $N00005                    0000000180007995     nframepop001.exp
 0002:000029c7       $N00006                    00000001800079c7     nframepop001.exp
 0002:00002a03       $N00007                    0000000180007a03     nframepop001.exp
 0002:00002a48       $N00008                    0000000180007a48     nframepop001.exp
 0002:00002a85       $N00009                    0000000180007a85     nframepop001.exp
 0002:00002acd       $N00010                    0000000180007acd     nframepop001.exp
 0002:00002b0d       $N00011                    0000000180007b0d     nframepop001.exp
 0002:00002b4a       $N00012                    0000000180007b4a     nframepop001.exp
 0002:00002b85       $N00013                    0000000180007b85     nframepop001.exp
 0002:00002bb3       $N00014                    0000000180007bb3     nframepop001.exp
 0002:00002be4       $N00015                    0000000180007be4     nframepop001.exp
 0002:00002c13       $N00016                    0000000180007c13     nframepop001.exp
 0002:00002c42       $N00017                    0000000180007c42     nframepop001.exp
 0002:00002c77       $N00018                    0000000180007c77     nframepop001.exp
 0002:0000307a       .idata$6                   000000018000807a     kernel32:KERNEL32.dll
 0002:000030de       .idata$6                   00000001800080de     vcruntime:VCRUNTIME140.dll
 0002:00003240       .idata$6                   0000000180008240     ucrt:api-ms-win-crt-runtime-l1-1-0.dll
 0002:00003262       .idata$6                   0000000180008262     ucrt:api-ms-win-crt-stdio-l1-1-0.dll
 0002:00003282       .idata$6                   0000000180008282     ucrt:api-ms-win-crt-string-l1-1-0.dll
 0003:00000000       ?codeAttributeName@@3PEBDEB 0000000180009000     libnframepop001.obj
 0003:00000008       ?lineNumberAttributeName@@3PEBDEB 0000000180009008     libnframepop001.obj
 0003:00000010       ?localVarAttributeName@@3PEBDEB 0000000180009010     libnframepop001.obj
 0003:00000018       ?localVarTypeAttributeName@@3PEBDEB 0000000180009018     libnframepop001.obj
 0003:00000020       ?stackMapAttributeName@@3PEBDEB 0000000180009020     libnframepop001.obj
 0003:00000028       ?callBytes@@3PAEA          0000000180009028     libnframepop001.obj
 0003:0000002c       ?allocBytes@@3PAEA         000000018000902c     libnframepop001.obj
 0003:0001aad4       redefineAttempted          0000000180023ad4     libnframepop001.obj
 0003:0001aad8       nsk_context                0000000180023ad8     libnframepop001.obj
 0003:0001aae4       redefineSucceed            0000000180023ae4     libnframepop001.obj
 0003:0001aae8       agentFailed                0000000180023ae8     libnframepop001.obj
 0003:0001aaec       currentAgentStatus         0000000180023aec     libnframepop001.obj
 0003:0001aaf0       context                    0000000180023af0     libnframepop001.obj
 0003:0001aba8       agentThread                0000000180023ba8     libnframepop001.obj
 0003:0001abb0       agentThreadProc            0000000180023bb0     libnframepop001.obj
 0003:0001abb8       agentThreadArg             0000000180023bb8     libnframepop001.obj
 0003:0001abc0       agent_data                 0000000180023bc0     libnframepop001.obj
 0003:0001abd0       jvmti_env                  0000000180023bd0     libnframepop001.obj
 0003:0001abd8       jvm                        0000000180023bd8     libnframepop001.obj
 0003:0001abe0       jni_env                    0000000180023be0     libnframepop001.obj
 0003:0001abe8       checkStatus_func           0000000180023be8     libnframepop001.obj
 0003:0001abf0       ?codeAttributeIndex@@3GA   0000000180023bf0     libnframepop001.obj
 0003:0001abf2       currFlag                   0000000180023bf2     libnframepop001.obj
 0003:0001abf3       popFlag                    0000000180023bf3     libnframepop001.obj
 0003:0001abf4       ?lineNumberAttributeIndex@@3GA 0000000180023bf4     libnframepop001.obj
 0003:0001abf8       ?localVarAttributeIndex@@3GA 0000000180023bf8     libnframepop001.obj
 0003:0001abfc       ?localVarTypeAttributeIndex@@3GA 0000000180023bfc     libnframepop001.obj
 0003:0001ac00       ?stackMapAttributeIndex@@3GA 0000000180023c00     libnframepop001.obj
 0003:0001ac04       ?stackFrameOffset@@3GA     0000000180023c04     libnframepop001.obj
 0003:0001ac08       ?mode@@3HA                 0000000180023c08     libnframepop001.obj
 0003:0001ac0c       ?constantPoolSize@@3GA     0000000180023c0c     libnframepop001.obj
 0003:0001ac10       ?orig@@3PEBEEB             0000000180023c10     libnframepop001.obj
 0003:0001ac18       ?gen@@3PEAEEA              0000000180023c18     libnframepop001.obj
 0003:0001ac20       ?inputPos@@3PEAEEA         0000000180023c20     libnframepop001.obj
 0003:0001ac28       ?endPos@@3PEBEEB           0000000180023c28     libnframepop001.obj
 0003:0001ac30       ?genPos@@3PEAEEA           0000000180023c30     libnframepop001.obj
 0003:0001ac38       ?markPos@@3PEAEEA          0000000180023c38     libnframepop001.obj
 0003:0001ac40       ?constantPool@@3PEAPEADEA  0000000180023c40     libnframepop001.obj
 0003:0001ac48       ?constantPoolCount@@3GA    0000000180023c48     libnframepop001.obj
 0003:0001ac4c       ?zeroBytes@@3PAEA          0000000180023c4c     libnframepop001.obj
 0003:0001ac50       ?codeLength@@3IA           0000000180023c50     libnframepop001.obj
 0003:0001ac54       result                     0000000180023c54     libnframepop001.obj
 0003:0001ac58       ?map@@3PEAIEA              0000000180023c58     libnframepop001.obj
 0003:0001ac60       ?widening@@3PEACEA         0000000180023c60     libnframepop001.obj
 0003:0001ac68       jvmti                      0000000180023c68     libnframepop001.obj
 0003:0001ac70       caps                       0000000180023c70     libnframepop001.obj
 0003:0001ac80       callbacks                  0000000180023c80     libnframepop001.obj
 0003:0001adb8       mid1                       0000000180023db8     libnframepop001.obj
 0003:0001adc0       mid2                       0000000180023dc0     libnframepop001.obj
 0003:0001adc8       currThread                 0000000180023dc8     libnframepop001.obj
 0003:0001add0       popThread                  0000000180023dd0     libnframepop001.obj
 0003:0001add8       currClass                  0000000180023dd8     libnframepop001.obj
 0003:0001ade0       popClass                   0000000180023de0     libnframepop001.obj
 0003:0001ade8       currMethod                 0000000180023de8     libnframepop001.obj
 0003:0001adf0       popMethod                  0000000180023df0     libnframepop001.obj
 0003:0001adf8       currLoc                    0000000180023df8     libnframepop001.obj
 0003:0001adfc       popLoc                     0000000180023dfc     libnframepop001.obj
 0003:0001ae10       GS_ExceptionRecord         0000000180023e10     MSVCRT:gs_report.obj
 0003:0001aeb0       GS_ContextRecord           0000000180023eb0     MSVCRT:gs_report.obj
 0003:0001b380       ?g_tss_cv@@3U_RTL_CONDITION_VARIABLE@@A 0000000180024380     MSVCRT:thread_safe_statics.obj
 0003:0001b388       ?g_tss_event@@3PEAXEA      0000000180024388     MSVCRT:thread_safe_statics.obj
 0003:0001b390       ?g_tss_mutex@@3U_RTL_CRITICAL_SECTION@@A 0000000180024390     MSVCRT:thread_safe_statics.obj
 0003:0001b3b8       ?g_sleep_condition_variable_cs@@3P6AHPEAU_RTL_CONDITION_VARIABLE@@PEAU_RTL_CRITICAL_SECTION@@K@ZEA 00000001800243b8     MSVCRT:thread_safe_statics.obj
 0003:0001b3c0       ?g_wake_all_condition_variable@@3P6AXPEAU_RTL_CONDITION_VARIABLE@@@ZEA 00000001800243c0     MSVCRT:thread_safe_statics.obj
 0003:0001b3cc       ?__proc_attached@@3HA      00000001800243cc     MSVCRT:dll_dllmain.obj
 0003:0001b3e0       ?is_initialized_as_dll@@3_NA 00000001800243e0     MSVCRT:utility.obj
 0003:0001b3e1       ?module_local_atexit_table_initialized@@3_NA 00000001800243e1     MSVCRT:utility.obj
 0003:0001b3e8       ?module_local_atexit_table@@3U_onexit_table_t@@A 00000001800243e8     MSVCRT:utility.obj
 0003:0001b400       ?module_local_at_quick_exit_table@@3U_onexit_table_t@@A 0000000180024400     MSVCRT:utility.obj
